:030000000219FDE5
:03000B000200A848
:03002B0002015A75
:03005B000202E5B9
:030073000202D2B4
:1000800002030406080C10182030406080040608A3
:100090000C10182030406080A0C00003070F1F051F
:1000A000050D050305030302C2AFC0D0C0E0206206
:1000B00014E5256009E473E525F4F58AD262D0E001
:1000C000D0D0D2AF3285268AC262E526F4602F30C6
:1000D000682520720DD0E0D0D0C2B1C287C281D2D3
:1000E000AF32C2B1C287C281206F0C206509740A89
:1000F000D5E0FDE57B4280D0E0D0D0D2AF32758A2A
:1001000000C28DD26201F701B7306805206502D2C6
:10011000B101B7306805206502D28701B7306805A4
:10012000206502D28101B7C28230680A2065077457
:1001300008D5E0FDD2B101B7C28630680A20650754
:100140007408D5E0FDD28701B7C28030680A206507
:10015000077408D5E0FDD28101B7C2AFC2AD53E646
:10016000EFC0D0C0E0D2D3D2AFC2CEE52A60072024
:100170007449152A21BB7800790020742EE580305F
:100180007E01F430E50278FF53DACF207E0343DAB4
:1001900020307E0343DA10C2D8C271E580307E0180
:1001A000F430E50279FFC3E89970CB306103752A1A
:1001B00018207403752A18885CD27020740DE52B02
:1001C0006004152B21CB43DA01C2D8207002413ED6
:1001D000A85C206102C270207431C3E894F040032F
:1001E00074F0F8E8C4540F28F87984B70302410B7F
:1001F000C313C3138721200802C313200A06C3C8F0
:1002000098F8410B28F8500374FFF8C3E89565503F
:1002100003E565F88822E52D54066022206B1FE572
:1002200036C333C333F8E564C313C313F9C395224C
:1002300040028922E82522F52250037522FF8522FB
:1002400024A824C3E52495614002A8618825E566B9
:1002500070024182C3E8AA669A5003E8FAE4F9EA18
:10026000C333FBE568F45B29400D2567F8E567605B
:10027000021567400B41820AC3E5679A5002056781
:1002800078FF8826C26FC3E52694F84002D26F201B
:10029000CF0AD0E0D0D043E610D2AD32C2CF053A7B
:1002A0007801E52A6005307402152AC3E55C9401E3
:1002B0004005755F0041C8756000756900E55F2401
:1002C00001F55F5003755FFFD0E0D0D043E610D258
:1002D000AD32C2AF53E67F7592FA7593FFC2607577
:1002E0009104D2AF32C2AF53E6EFC2ADC0D0C0E08E
:1002F000C0F0D2D3D2AFA8FBA9FCC2D83071026142
:100300004C53DACF207E0343DA10307E0343DA20E9
:10031000D271E580307E01F420E5026123882789CF
:1003200028A17953DACF207E0343DA20307E0343BD
:10033000DA10C2D8C271307402A1657800E580304D
:100340007E01F430E502A165885CA14D53DACF202F
:100350007E0343DA20307E0343DA10C2712061024B
:10036000812553DACF207E0343DA10307E0343DA4F
:1003700020C2D8D27188578958C3E89555F8E995B5
:1003800056F97B007E087A00C3E8948CE99400500B
:1003900005755B008117882178A2E6A8216055C306
:1003A000E894C8E994005008E4D2E4FB7A0A61F2C8
:1003B000C3E89468E994015008E4D2E3FB7A0F6142
:1003C000F2C3E894D0E994025008E4D2E2FB7A1E2A
:1003D00061F2C3E894A0E994055008E4D2E1FB7A05
:1003E0003C61F2C3E89498E994085008E4D2E0FB39
:1003F0007A787E00C3E89559FCE9955AFD30E70A02
:10040000ECF42401FCEDF43400FD755B00C3EC9AC0
:10041000ED9E5003755B018859895A85575585585B
:10042000567802A14DC3E89527F8E99528F9307C64
:1004300002A131307B02A131307A02A12A2075025B
:100440008148E9FDE8FC8167E9C313F9E813F83056
:100450007902A12AE9C313F9E813F8307802A12A36
:10046000E9C313FDE813FC20612CC3EC941CED944C
:0E047000024002817EED701EC3EC94C850184D
:10047E000529E52970021529C3E529940A5002A120
:10048E0065755C00D270A165E52960021529788832
:10049E00E6F97400207F087896B90302789EE62468
:1004AE00FAFEE43400FFC3EC9EFCED9FFD9208B90A
:1004BE000310A2085007207609D27681D03076023A
:1004CE00C276A2085016B9030DECF42401FCEDF42B
:1004DE003400FD0204EA78007900A131B90315EC6D
:1004EE0033FCED33FDC3EC940AFCED9400FD500497
:1004FE007C007D00C3EC94FFED9400400678FF79FC
:10050E0000A131EC8572F0A4C5F0A2F733F87900A2
:10051E00400302054D78FF790002054DE9C313F93A
:10052E00E813F8307C0EE9600278FFC3E81338F860
:10053E00E43400F9C3E894FFE99400400278FF88A0
:10054E005CD270206102A165741FF4552F4BF52FFC
:10055E00C274EB7002D274752A18307403752A0AAD
:10056E00306102A17920740353DAFE207403752BD7
:10057E0006D0F0D0E0D0D0D2AD43E61032790102F1
:10058E0005A979030205A9790A0205A9791E0205B2
:10059E00A979640205A979C80205A97817E4D5E0FE
:1005AE00FDD8FAD9F6227A147B780205D07A107B20
:1005BE008C0205D07A0D7BB40205D07A0B7BC80273
:1005CE0005D0E573D5E001227902E4C286D5E0FDBF
:1005DE00D287D5E0FDC287D5E0FDD286D5E0FDE914
:1005EE0020E002D2B130E002D281E573D5E0FDE920
:1005FE0020E002C2B130E002C2817496D5E0FDD98E
:10060E00C9EAF8D5E0FDD8FBDBB8C28622C37C0070
:10061E007D0075F00005F0EA33FAEB33FB50F6EB94
:10062E0013FBEA13FAC3E9FFE8FEE89AF8E99BF92F
:10063E005004EFF9EEF8B3EC33FCED33FDD5F0DFFB
:10064E00EDF9ECF822E889F08A20D2D4F8A9F07BF3
:10065E000030F70B7BFFF42401F8E9F43400F9E8DD
:10066E008520F0A4ADF0F8E98520F0A4AFF0FEED02
:10067E002EF974003FFA7C04C3EA13FAE913F9E881
:10068E0013F8DCF48BF030F70AE8F42401F8E9F4FF
:10069E003400F9E889F0C2D4F8A9F02222C3E5416A
:1006AE0013F9E54013F8C3E54498F8E54599F95078
:1006BE000CC3E89480E994FF40160206E2C3E89466
:1006CE007FE9940050030206E2787F79000206E289
:1006DE00788079FF8849894A22E5492546F8E54A16
:1006EE003547F9854A20E4300701F43548FA30E7FA
:1006FE0009C3EA94F04015020720C3EA940F500391
:10070E0002072078FF79FF7A0F0207207800790020
:10071E007AF0C3E5249561500AC374019524500BF9
:10072E0002073EE54A20E70E02073EE54A30E7069D
:10073E00884689478A482278A5E6FAC3E54933F800
:10074E00E54A33F9D153E930E70BC3E89480E994D5
:10075E00FF4013E178C3E8947FE994005002E178FA
:10076E00787F7900E178788079FFE820E715C3E596
:10077E002398F84009C3E89401400302079F7801CB
:10078E0002079FE8F424012523F8400302079F780F
:10079E00FF884B2278A6E6FAA847A948D153E9303C
:1007AE00E70CC3E89401E994FF40160207D3C3E8AF
:1007BE0094FFE9940050030207D378FF79000207F3
:1007CE00D3780179FFE920E715C3E54B98F8400986
:1007DE00C3E8940140030207FA78010207FAE8F42D
:1007EE002401254BF840030207FA78FF882422786B
:1007FE00FF20692879A1E76023E541601F74FF851A
:10080E0041F0848539F0306A0375F005A4F8C5F01F
:10081E00600278FFC3E895645002A864886322C31F
:10082E00E5409440E5419401E563500314013E0414
:10083E006002F563220208462275E890227883E66C
:10084E00FF30EDF9A8BDA9BE0570C3E57094084050
:10085E0052757000E9FA79A0E76044EA7007E57115
:0F086E00601B02087FC3E895716010E5715006AA
:10087D00600C1402088B0460F902088BE571F571A8
:10088D00C394A8401B7561C0C39405401375618066
:10089D00C39405400B756140C39405400375610019
:1008AD0075BB0622E561F460020561E570B40703CE
:1008BD0075BB1E22743279A787F0A4C5F0A2F73359
:1008CD00F8C3E895614002A86188228824882588AC
:1008DD00268864227540007541F022C2AF75C8208C
:1008ED00A8CCA9CDAA3A30CF010A75C824D2AFAB96
:1008FD003BAC3C883B893CC3E89BF8E99C206908EC
:10090D00F930660221F72151AD3D8A3DF9EA9DFA94
:10091D00600478FF79FFAE3EAF3F8B3E8C3FA83B26
:10092D00A93CC3E89EF8E99FF9C3E54113FBE540F7
:10093D0013FAE82AF540E93BF54150067540FF757D
:10094D0041FF219EAA40AB41AC40AD417E047F02E8
:10095D00C3EB9404400D1E1FC3EB94084005206AA1
:10096D00021E1FC3ED13FDEC13FCDEF7C3EA9CFA68
:10097D00EB9DFBEF6009C3E913F9E813F8DFF7EA24
:10098D0028FAEB39FB8A408B4150067BFF8B408B5D
:10099D0041C3EB94025002D2663069047F0321C932
:1009AD007892E6FFC3E537948240110FC3E5379483
:1009BD00A040010FC3EF940640027F057E02E54182
:1009CD00C4540FF9E541C454F0F8E540C4540F2860
:1009DD00F8C3E89EFAE99400FB4009C3EA9402EBE0
:1009ED00940050047A02E4FB4143AA40AB41EBC4AE
:1009FD00FEEAC4540F4EFCC3EA9CFAEB9400FBC311
:100A0D00E813C313F8EA28FAEB3400FB8A408B4154
:100A1D00C3EB94024002C2667802EBC4FE7B00EA8F
:100A2D00C4540F4EFAC3EA98FA4005C3940250021B
:100A3D007A027892E6FF30600241438551928552E9
:100A4D0093D26043E680C3E49AF8E49BF9306602E2
:100A5D0041CFE8FAE9FBD3E913FDE813FC8851898E
:100A6D0052C3EF94036038EF20E00DE82CF8E93D18
:100A7D00F9ECFAEDFB020A98E828F8E939F9C3E830
:100A8D002402F8E93400F97AFE7BFFC3EF940340AA
:100A9D000E8A538B54884D894E8C4F8D506103882F
:100AAD005389548A4D8B4E8C4F8D5030691275532E
:100ABD00F07554FF754FF07550FF7551F07552FF7D
:100ACD006103E8FAD3E813FC8851C3EF9403602067
:100ADD00EF20E007E82CF8ECFA41EFE8282402F8C3
:100AED007AFEC3EF940340088A53884D8C4F6103FF
:100AFD0088538A4D8C4FE568C3335002646BF5689B
:100B0D00306002610D753402D26043E680E52D54EC
:100B1D00066034A840A941C3E913F9E813F8C3E905
:100B2D0013F9E813F8306904E92440F9C2AF53E62C
:100B3D007F759100C3E498F594E499F5957591044A
:100B4D00D26043E680D2AF22D26475430075200097
:100B5D00306C03752040020B74D264754300752010
:100B6D0040306C0375200078017901206620E52D59
:100B7D0054066002C2647914E541C313700104F890
:100B8D00C3941440027814306904781B791B2060DB
:100B9D0010E543600C306903D53404D26D811E71AC
:100BAD00150543E59B5440B52002810830690908BD
:100BBD00C3E899400118619B20640A08C3E8994075
:100BCD00026174619BC264C2AF53E67F75910030C0
:100BDD0066127594007595F8759104D26043E680A0
:100BED00D2AF6174E5417EFFC3334005C33340018D
:100BFD00FEC3E49E759400F59561E5C3E53394015C
:100C0D00500261743064026174D802811C619BC210
:100C1D006DC2AF53E67F75910085539485549575DC
:100C2D009104854D92854E93D26043E680D2AFE517
:100C3D002D54066008206A020533020C5A306D0DE2
:100C4D00206C0A2064071581158102153822780061
:100C5D003064027801E53775F007A4F9E5F028F561
:0E0C6D00F0E9A2F013A2F113A2F213F537C3BF
:100C7B0094785003753778C3E53795384008D265BB
:100C8B00C2B1C287C2813060028191854F9285507B
:100C9B0093D26043E68022207D16C2AF754202C21A
:100CAB0086D282306202D281D2AF759F02020E9140
:100CBB00C2AF754202C286D280306202D2B1D2AFCD
:100CCB00759F02020E91307243207D20C2AF754298
:100CDB0003900138757B40C281C280306204D28799
:100CEB0081EFD286D2AF759F03020E91C2AF7542D0
:100CFB0003900138757B40C2B1C282306204D28747
:100D0B00A10FD286D2AF759F01020E91207D17C223
:100D1B00AF754203900113C281306202D287D2AF0A
:100D2B00759F03020E91C2AF754203900113C2B1BE
:100D3B00306202D287D2AF759F01020E91207D16D1
:100D4B00C2AF754204C282D280306202D287D2AF68
:100D5B00759F01020E91C2AF754204C280D28230E0
:100D6B006202D287D2AF759F03020E91307243207D
:100D7B007D20C2AF754205900127757B04C287C2E7
:100D8B0086306204D2B1A195D282D2AF759F020296
:100D9B000E91C2AF754205900149757B01C287C2A6
:100DAB0086306204D281A1B5D280D2AF759F020288
:100DBB000E91207D17C2AF754205900109C2873095
:100DCB006202D2B1D2AF759F02020E91C2AF7542D1
:100DDB000590011DC2873062EBD281D2AF759F02A5
:100DEB00020E91207D16C2AF754206C280D28630AC
:100DFB006202D2B1D2AF759F03020E91C2AF7542A0
:100E0B0006C282D286306202D281D2AF759F0102B6
:100E1B000E91307243207D20C2AF75420190014983
:100E2B00757B01C2B1C282306204D281C13BD280D8
:100E3B00D2AF759F01020E91C2AF7542019001278F
:100E4B00757B04C281C280306204D2B1C15BD28295
:100E5B00D2AF759F03020E91207D17C2AF75420171
:100E6B0090011DC2B1306202D281D2AF759F0102D7
:100E7B000E91C2AF754201900109C281306202D25C
:100E8B00B1D2AF759F03C26522900107757B00C27B
:100E9B00B1C287C281C282C286C280C262227880FE
:100EAB0076FF0876FF0876FF0876FF08760308764C
:100EBB0004087609087603087601087601788C76A3
:100ECB00010876FF0876FF0876FF0876FF0876FFA5
:100EDB000876030876FF0876FF0876FF0876250864
:100EEB0076D00876FA0876FA0876040876FF087644
:100EFB000108760008767A0876FF087601087601F5
:100F0B00087600087603087600227887E6FFC2721F
:100F1B00BF0302D2727888E6C394036008C27DE6F1
:100F2B0030E102D27DC27E7889E630E102D27EC307
:100F3B00EF94026008758E01D273020F4D758E000F
:100F4B00C273227880E6149000809378A5F678819E
:100F5B00E6149000809378A6F67886E61490008DC0
:100F6B009378A7F67886E6F539C394025003753962
:100F7B0002789CE67538FFB402037538A0B40303FE
:100F8B0075388278A3E61490009A93F566D1942273
:100F9B00C2B3789DE66002D2B3227896E6FA7897D0
:100FAB00E6FB7888E6B40305C3EB940EFB307F04B5
:100FBB007A007BFFC3EB9AFCC3948250027C827550
:100FCB0072000572EC8572F0A4C3E5F0947D40F2DB
:100FDB0022D27FF1A512059A12059A7A007B007C2A
:100FEB0010120590E55C2AFA74003BFBDCF37C04E1
:100FFB00C3EB13FBEA13FADCF7FEC27F120FA52239
:10100B00757C00757D00E5EF20E60375200005205B
:10101B00903DFFE520146006901FFF1460009304C1
:10102B00600375EF1653D9BF7581C043FF8012055E
:10103B008B75EF0643B203E5B3240220E70DF521D0
:10104B00E5B120E0068521B343B101120E94758002
:10105B003875A4C775F1FF75D4DF7590FF75A500C2
:0F106B0075F20075D50075A0FF75A60075F3002E
:10107A0075D60075B0E475A71B75F4FF75E24112C9
:10108A000E94E4F8F6D8FD756801120EA9121589B6
:10109A0078988673753001C2AF1205A41205B4128E
:1010AA00059A1205BB12059A1205C212059A121662
:1010BA00A61205A41205A412059FC2AF757C00757D
:1010CA007D0078FA79FA308507D9FBD8F7021C0037
:1010DA00120F15120F4E120F9B120FA578988673D6
:1010EA00120E9475881075890275C8247591047555
:1010FA00D84075A82275B80275E690759B80759DD3
:10110A000075D10E75BC5875BB0675BA1F75E88097
:10111A0012058BD2AF12084375360053DACF207E00
:10112A000343DA20307E0343DA1043DA01C2D8C21D
:10113A00711205A4D2617B037A0CE55B70077A0C05
:10114A00DB030210C412059A2070030210C4C27095
:10115A00E55CC3940240E1E52F541F855E5DF55EB0
:10116A00B55DD5DAD5C26153DACF207E0343DA20E2
:10117A00307E0343DA10C2D8C27178A2E67008D270
:10118A0074E52F54E0F52FC27575290012059F30BA
:10119A007409C3E529940A4002D2751205907802AF
:1011AA003074027800C3E55C9840F0C2AF1205B40F
:1011BA001205B41205B4D2AF1205A4754C00788892
:1011CA00E6B4030241C4120590788CE6C394015038
:1011DA00030212C4E530C3940150030212C4757CA1
:1011EA00A5757DF1207435C3E55C94FF50030212A6
:1011FA00C4C2AF1205C9D2AF12059FC3E55C940100
:10120A0050EFC2AF1205B41205951205B4D2AF124F
:10121A00059FC3E55C94FF40E902172B7F05D27F47
:10122A00120FA512059FC2AFC27F120FA5AE5CC3F3
:10123A00E55C947FD2AF500241D412058BC2AF1243
:10124A0005C9D2AFDFD8120FDCC3EE94057897F642
:10125A001205A41216AE7F0AD27F120FA512059F9D
:10126A00C2AFC27F120FA5AE5CC3E55C947FD2AF5A
:10127A0050E412058BC2AF1205B41205951205B4DB
:10128A00D2AFDFD4120FDCEE24037896F6F8799702
:10129A00E7C394824003985006E824827897F612AE
:1012AA0005A41215CB1216DD12059F120FA5C3E570
:1012BA005C94FF500221E802172B757C00757D00B3
:1012CA00C3E55C954C4003855C4C12059F78017917
:1012DA0088E7B403027805C3E55C98400221C8C2D6
:1012EA00AF1205C91205C91205C9D2AF1205A475F4
:1012FA003000E4F531F5320531E531F4703F05325D
:10130A00789AE67819146012783214600D787D1490
:10131A00600878FA146003753200C3E53298401DFC
:10132A00120E9412058B153275310078998673C2A4
:10133A00AF1205C9D2AF7898867312059F12059528
:10134A00E52A700530740201C47801207402780617
:10135A00C3E55C9840A17888E6C39403600312054C
:10136A009FE52A70030210C4C2AF120E94E4F5225C
:10137A00F523F524F525F526F567D2AF7885E6C37A
:10138A0033F565E4F544F545F546F547F548F57056
:10139A00F52CF52DF53775700875BB1E12058B12E5
:1013AA00084730EDFDA8BDA9BEE97001F8887112A1
:1013BA00084B75700875BB1E120F15C2AF7561FF19
:1013CA001208C1852261852262852263D2AF752205
:1013DA0001752401752501752601856069756A0103
:1013EA007888E6B40307C27D307602D27DD268D20D
:1013FA0069753300120DEE120E1D1208E11208E88B
:10140A001208E11208E81208E1120B661206AA1283
:10141A000C5B120CA21208E8120B55306E0312066E
:10142A00AB2066031207FD30660312082D120C5B0F
:10143A00120CD11208E8120B66306E031206E7127C
:10144A000C5B120D481208E8120B55306E03120796
:10145A0045120C5B120D771208E8120B66306E0308
:0F146A001207A2120C5B120DEE1208E8120847CF
:10147900120B55120C5B120E1D12084B1208E830A4
:10148900692F856461856462856069756A01791867
:101499007A0CC3E53399400CC269D26A8A35756101
:1014A900FF0214BAC3E55C94014003021413021548
:1014B90040306A1D206C1AE535147006C26AD26B79
:1014C9008113F535C3E55C94014003021413021539
:1014D90040753600788279A4E760027803C3E55F36
:1014E900985054307404E52A604D7888E6B403179F
:1014F900207D05207607A110307602A110206C0707
:10150900D26C856461815278F0306C0585646178AC
:1015190020C3E5419850028113306C1BC26CC27D17
:10152900307602D27DD26A753512856461811305E0
:1015390036E55C6002A143753600C2AF120E94789D
:1015490087E6FE7602120F157887EEF6E4F522F5A6
:1015590023F524F525F526F565752C00752D00D2A2
:10156900AF12059F120E9478A4E66006D2B1D28715
:10157900D281307409C3E5369404400201C441FCA8
:10158900901A0D782012160DE520B45A0CA31216E4
:101599000DE520B4A5030215AB120EA91215CB0255
:1015A90015CA901A0378807B0A12160DA308DBF975
:1015B900901A0F788C7B1912160DA308DBF9901A73
:1015C9002822C2AF12165012162D901A00740E124C
:1015D9001612A37407121612A37415121612901A72
:1015E9000378807B0A121611A308DBF9901A0F7889
:1015F9008C7B19121611A308DBF912166312164116
:10160900901A2822E493F622E6438F01538FFDFFB7
:10161900C3E583941C400122EF857CB7857DB7F033
:10162900538FFE22438F02438F01857CB7857DB797
:10163900901A0DF0538FFC22901A0D745AD1129002
:101649001A0E74A5D112227A3079D07820901A40D6
:10165900D10DE520F709A3DAF7227A3079D0901A6B
:1016690040E7D11209A3DAF922AB74A875BB0102CC
:101679007984BB02027985BB03027986BB040279AE
:1016890092BB05027987BB060279A3BB0702799C45
:10169900BB08027988BB09027989E8F7227C05121F
:1016A90005A4DCFB22C2AF1205B41205BB1205C2A8
:1016B9001205C91205951205B41205BB1205C2120D
:1016C90005C91205951205B41205BB1205C212050A
:1016D900C9D2AF22C2AF1205C91205C21205BB1287
:1016E90005B41205951205C91205C21205BB1205EA
:1016F900B41205951205C91205C21205BB1205B42B
:10170900D2AF22AE74AF75C2AF1205B41205B412CE
:1017190005B4120595DEF21205C9120595DFF8D256
:10172900AF22D1AED1A6D1A67574017575017576B2
:1017390000F10C7C05AD5C1205A4C3ED955C70F558
:10174900C3E55C9401400AC3E55C94FF403202178B
:1017590067D172B1CBD1AEC2AF75EF16D1A6DCD5C8
:101769000576C3E5769403500280C6D1A60575E5D2
:10177900741490009F93F808C3E57598500280AEE1
:10178900D1A6D1A60574C3E574940A5002809C12AF
:0B1799000EA9B1CBC2AF75EF16D1A6B0
:0319FD0002100BCA
:101A00000E0715FFFFFFFF0304090301015AA5019B
:101A1000FFFFFFFFFF03FFFFFF25D0FAFA04FF01DE
:091A2000007AFF0101000300FF40
:101A4000235475726E6967794145343541232020EE
:101A500023424C48454C4923463331302320202033
:101A60002020202020202020202020202020202076
:101C0000C2AFC2D353D9BF7581C043B20343FF8073
:101C1000752438752503B1DC7529A5752AF175E29F
:101C20004043F12053A4DF75D4FFD2857DFA7803B9
:101C300079E67C10752200752300901DE97B0675FE
:101C400024987525013085028145208508D8FBD967
:101C5000F9DCF781B7308508D8FBD9F9DCF781B713
:101C6000B19CE493A3C39A6004DDC381B7DBDBB10D
:101C70008E6002812E7B08E493FAA3B16FDBF87AC1
:101C800030B16F752200752300B18EEAFCEBFDC305
:101C9000ED94FE400EB18E8A278B28ED30E0048A49
:101CA000828B83B18E7AC270D8C3ED94FE601950D6
:101CB000CEBD002BEC600F7520007521FF7529004B
:101CC000752A000200008100A827A9280809D80465
:101CD000D90281DCB192EA89AAF281CE0D81A3C337
:101CE000ED94035053EDA2E092007AC5C3E58294CF
:101CF00000E583941C508A200010438F02438F011B
:101D00008529B7852AB7F0300029A827A92808090E
:101D1000438F01538FFDD804D902A133C3E58394C7
:101D20001C4003A3A11689AAE28529B7852AB7F02A
:101D3000A3A116538FFC817F7AC1BD030CE493A34A
:101D4000FAB153DCF8B14B817F8181AA22AB23B178
:101D50006FEBFAEA6222752608C3E52313F523E543
:101D60002213F52250066323A0632201D526EAB18F
:101D7000DCB1DC75260AEAF4200102D285300102CA
:101D8000C285B1DCC3134002C201D526EB22B19259
:101D9000EAFB208502A192308502A197752608AE44
:101DA00024AF25C3EF13FFEE13FEB1E0B1DCC3EAAD
:101DB000133085024480FA30E703632201C3E52330
:101DC00013F523E52213F52250066323A0632201B5
:101DD000D526D9E52265236523F52222AE24AF2539
:101DE0000E0FDEFEDFFCD20122424C48656C6934E6
:071DF000373163F310060117
:00000001FF
